:100000008D2964001720031801285620A801083004
:10001000A300572017200318A80AAB1EA801A20CA2
:10002000A30B0928AB1AA2135720220808003A088C
:100030008400380884178004841300052B1B3806BD
:10004000FF3E08000408A6003A088400F030B70517
:100050000830A70003100318B70A3C20A60CA70B12
:100060002B280000AB1A370C3C208B2103143C20BA
:100070002F08A3002E08EC288413AB1F4B28000880
:1000800038042B1F38068000841700083804031C2E
:1000900038068000572800083804031C38062B1B3C
:1000A00038068000841738098005572837172B0831
:1000B0001F39FF3EA1002A08F53E0318A10A371F89
:1000C000F9283713A00002302B21F928B71329088B
:1000D0000319B7170530A8002730A30010307C2083
:1000E0000330A300E8307C20A30164307C20A3010E
:1000F0000A307C2024088328A2002508A1002408B7
:10010000A00051212008A000A8030319B713290853
:1001100003198D282802031808002008031DB713AF
:10012000B71B0800303E83290830A60037180D2180
:100130003B08840039083719B720371DB9203A0821
:1001400084003809BD203A088400A10CA00C0008E6
:100150003804031C38068000B020A60BA328882989
:100160003B088400390880060000800608008004EF
:10017000BC28FF3A8005BD28FF3A841780058829EE
:10018000A000A00DA00DA00D3830A00581302004E6
:100190009F000030A1003230F9201F151F19CE2812
:1001A0001E08A10083161E08882903178D008316D8
:1001B0008C130C1483120C08882903178C008316E7
:1001C0008C130C1555308D00AA308D008C148C18B2
:1001D000E7280C118829A301A200FF30A207031C05
:1001E000A307031C88290330A100DF30F920ED2884
:1001F000A101E83EA000A109FC30031C0229A007D0
:100200000318FF28A0076400A10FFF282018082961
:10021000A01C0C2900000C290800A400A201A301C5
:100220001529A10CA00CA20DA30DFF3E0318112946
:10023000240823212208A0042308A1042008080080
:100240000310A00DA10DFF3E0318202920088829C6
:100250000310A10CA00CFF3E0318282920088829B0
:10026000A101A301A20001303A29A101A301A2002A
:1002700004303A29A80023082102031D412922083D
:100280002002043003180130031902302805031D31
:10029000FF3088290038031DFF300405031DFF309F
:1002A00088291030A600A501A401210DA40DA50DDB
:1002B0002208A4022308031C230FA50203186729A0
:1002C0002208A40723080318230FA5070310A00D75
:1002D000A10DA60B5529200888291030A800A101DE
:1002E000A001A70CA60C031C7B292208A007230849
:1002F0000318230FA107A10CA00CA50CA40CA80B9C
:10030000712924088829840031088A003008820075
:100310008313031383126400080083161F308500C3
:10032000013086008701831281309F00831684305C
:100330009F008312E330E600C4010230C5000712BB
:10034000831607128312861383168613831287116E
:100350008316871107308312BA000230B800543078
:10036000AA004030AB00AE01AF0120308A0123204B
:1003700050308A01232069308A01232063308A01AA
:1003800023202D308A01232054308A01232072300B
:100390008A01232061308A0123206E308A012320C4
:1003A00073308A01232063308A01232065308A015B
:1003B000232069308A01232076308A01232065308A
:1003C0008A01232072308A01232020308A012320D1
:1003D00056308A01232048308A01232046308A0182
:1003E000232020308A0123202D308A012320203031
:1003F0008A01232045308A01232041308A012320AD
:1004000033308A01232043308A0123204E308A0171
:1004100023204F308A01232020308A0123200A30F4
:100420008A0123200D308A0123200330A300E83005
:100430008A01EC2000308A01D520E40001308A01D5
:10044000D520E50002308A01D520EA0003308A0178
:10045000D520E90004308A01D520E20005308A0168
:10046000D520E7006408A600A7016430A200A3011C
:100470008A016D21B2002508B30065083207C60065
:1004800033080318013EC7004608A0004708A10032
:100490002A30A30048308A0132218A110A12031D32
:1004A000BD2E8A150A12952587158316871183128A
:1004B0008A150A1272268715831687110730831250
:1004C000BA000230B8005430AA004030AB00AE0190
:1004D000AF012A308A0123204D308A012320653064
:1004E0008A0123206E308A01232075308A0123205F
:1004F00020308A01232052308A01232058308A017B
:1005000023202A308A01232020308A0123206630CC
:100510008A0123203D308A01232046308A0123208E
:1005200072308A01232065308A01232063308A01DA
:1005300023202E308A01232020308A012320683096
:100540008A0123203D308A01232031308A01232073
:1005500030308A01232030308A0123204B308A0139
:10056000232048308A0123207A308A01232020303A
:100570008A0123206C308A0123203D308A01232008
:1005800031308A01232032308A0123202E308A0123
:10059000232035308A0123204B308A012320483024
:1005A0008A0123207A308A01232020308A012320E7
:1005B0006E308A0123203D308A0123206E308A016B
:1005C000232069308A01232076308A012320653078
:1005D0008A0123206C308A01232020308A012320C5
:1005E00071308A0123203D308A01232073308A0133
:1005F000232071308A01232075308A0123202E3078
:100600008A01232020308A01232073308A0123208D
:100610003D308A01232054308A01232058308A013A
:1006200023202D308A01232036308A0123203030C8
:100630008A01232030308A01232020308A012320A0
:1006400074308A0123203D308A01232054308A01EE
:10065000232058308A01232020308A01232076303D
:100660008A0123203D308A01232076308A0123200D
:100670006F308A0123206C308A01232075308A0173
:1006800023206D308A0123202E308A0123200A3056
:100690008A0123200D308A012320C8308A01EB20F3
:1006A0000730BA000130B8005430AA004030AB0027
:1006B0008A010120E8006808A00067308A0135211E
:1006C000B2006808A00065308A013021B400320809
:1006D000840034088A014A218A110A12031D292F35
:1006E0006808A00069308A013521B2006808A000BE
:1006F00067308A013021B4003208840034088A014E
:100700004A218A110A12031D052C6808A0006D30C9
:100710008A013521B2006808A0006B308A013021BF
:10072000B4003208840034088A014A218A110A126E
:10073000031D212D6808A0006F308A013521B20009
:100740006808A0006D308A013021B40032088400AE
:1007500034088A014A218A110A12031D3F2E6808B3
:10076000A00072308A013521B2006808A000703004
:100770008A013021B4003208840034088A014A21F9
:100780008A150A12031DAF286808A00074308A0178
:100790003521B2006808A00072308A013021B4000F
:1007A0003208840034088A014A218A150A12031D7E
:1007B000F42C6808A00075308A013521B200680861
:1007C000A00073308A013021B4003208840034085C
:1007D0008A014A218A150A12031D9B296808A00074
:1007E00077308A013521B2006808A00075308A018F
:1007F0003021B4003208840034088A014A218A1169
:100800000A12031DC62F8A015B2A0730BA00023084
:10081000B8005430AA004030AB00AE01AF01463002
:100820008A01232072308A01232065308A01232027
:1008300063308A01232075308A01232065308A01C4
:1008400023206E308A01232063308A0123206930FF
:100850008A01232061308A01232020308A0123204D
:100860002D308A01232020308A0123200230A90064
:100870006308A400A5012230B000B1018A016620FE
:100880000430A9003E08A4003F08A5002230B000B3
:10089000B1018A0166202E308A0123200130A9008F
:1008A0004008A4004108A5002230B000B1018A012F
:1008B00066204D308A01232048308A0123207A3077
:1008C0008A01232020308A01232020308A0123201E
:1008D0002B308A0123202F308A0123202D308A01DA
:1008E000232020308A01232031308A012320303018
:1008F0008A01232030308A01232020308A012320DE
:100900004B308A01232048308A0123207A308A0123
:10091000232020308A01232020308A0123206D30BB
:100920008A0123203D308A0123204D308A01232073
:1009300065308A0123206E308A01232075308A01B8
:1009400023200D308A0123200730BA000130B8007F
:100950005430AA004030AB008A010120E800FA3090
:100960008A01EB206808A0002C308A013521B200F2
:100970006808A0002A308A013021B40032088400BF
:1009800034088A014A218A110A12031DF32C6808CF
:10099000A0002E308A013521B2006808A0002C305A
:1009A0008A013021B4003208840034088A014A21C7
:1009B0008A110A12031D092D6808A0006E308A01F1
:1009C0003521B2006808A0006C308A013021B400E3
:1009D0003208840034088A014A218A110A12031D50
:1009E0005B2A8A01052C4608A0004708A1002A308E
:1009F000A30040308A0132218A110A12031D052CFE
:100A00000830C6070318C70A8A150A1295258A01F5
:100A1000052C4608A0004708A1002930A300B030EB
:100A20008A0137218A110A12031D052C0830C602DB
:100A30000030031C013EC7028A150A1295258A015F
:100A4000052C0730BA000230B8005430AA004030FC
:100A5000AB00AE01AF0146308A01232072308A011B
:100A6000232065308A01232063308A0123207530DA
:100A70008A01232065308A0123206E308A012320D9
:100A800063308A01232069308A01232061308A0182
:100A9000232020308A0123202D308A01232020307A
:100AA0008A0123200230A9006308A400A501223096
:100AB000B000B1018A0166200430A9003E08A400FC
:100AC0003F08A5002230B000B1018A0166202E3017
:100AD0008A0123200130A9004008A4004108A50094
:100AE0002230B000B1018A0166204D308A012320F6
:100AF00048308A0123207A308A01232020308A015D
:100B0000232020308A0123202B308A0123202F30FC
:100B10008A0123202D308A01232020308A012320BE
:100B200031308A01232032308A0123202E308A017D
:100B3000232035308A01232020308A0123204B30A6
:100B40008A01232048308A0123207A308A01232019
:100B500020308A01232020308A0123206D308A0131
:100B600023203D308A0123204D308A012320653027
:100B70008A0123206E308A01232075308A012320C8
:100B80000D308A0123200730BA000130B8005430FC
:100B9000AA004030AB008A010120E800FA308A0147
:100BA000EB206808A0002C308A013521B2006808CB
:100BB000A0002A308A013021B400320884003408B1
:100BC0008A014A218A110A12031D122E6808A00008
:100BD0002E308A013521B2006808A0002C308A012D
:100BE0003021B4003208840034088A014A218A1175
:100BF0000A12031D272E6808A0006E308A013521D5
:100C0000B2006808A0006C308A013021B4003208BC
:100C1000840034088A014A218A110A12031D5B2AC2
:100C20008A01212D4608A0004708A1002A30A30010
:100C300047308A0132218A110A12031D212DC60A6A
:100C40000319C70A8A150A1295258A01212D46081B
:100C5000A0004708A1002930A300A9308A0137214C
:100C60008A110A12031D212D0130C6020030031C17
:100C7000013EC7028A150A1295258A01212D0030EE
:100C80008A01C020C2002108C3004208A600430810
:100C9000A7000A30A200A3018A016D21B200250835
:100CA000B3003208A0003308A1004C30A200A30119
:100CB0008A015121B2002108B3003208853CBC00F2
:100CC0003308031C013E003CBD000730BA0002306F
:100CD000B8005430AA004030AB00AE01AF014E3036
:100CE0008A01232069308A01232076308A0123205B
:100CF00065308A0123206C308A01232020308A014C
:100D000023200330A9003C08A4003D08A5002230A0
:100D1000B000B1018A01662020308A0123206430AE
:100D20008A01232042308A0123206D308A0123204A
:100D30000D308A0123200730BA000130B80054304A
:100D4000AA004030AB008A010120E8006808A0003A
:100D50006E308A013521B2006808A0006C308A012B
:100D60003021B4003208840034088A014A218A11F3
:100D70000A12031D5B2A8A013F2EF830C600293073
:100D8000C7008A150A1295250730BA000230B8004C
:100D90005430AA004030AB00AE01AF0146308A01AA
:100DA000232072308A01232065308A01232063309A
:100DB0008A01232075308A01232065308A0123208F
:100DC0006E308A01232063308A01232069308A0132
:100DD000232061308A01232020308A0123202D30F6
:100DE0008A01232020308A0123200230A9006308D1
:100DF000A400A5012230B000B1018A0166200430B0
:100E0000A9003E08A4003F08A5002230B000B101AF
:100E10008A0166202E308A0123200130A900400873
:100E2000A4004108A5002230B000B1018A0166206B
:100E30004D308A01232048308A0123207A308A01EC
:100E400023200A308A0123200D308A0123208A01C1
:100E50005B2A0730BA000230B8005430AA00403094
:100E6000AB00AE01AF0146308A01232072308A0107
:100E7000232065308A01232063308A0123207530C6
:100E80008A01232065308A0123206E308A012320C5
:100E900063308A01232069308A01232061308A016E
:100EA000232020308A0123202D308A012320203066
:100EB0008A0123200230A9006308A400A501223082
:100EC000B000B1018A0166200430A9003E08A400E8
:100ED0003F08A5002230B000B1018A0166202E3003
:100EE0008A0123200130A9004008A4004108A50080
:100EF0002230B000B1018A0166204D308A012320E2
:100F000048308A0123207A308A01232020308A0148
:100F1000232020308A01232020308A0123206D30B5
:100F20008A0123203D308A0123204D308A0123206D
:100F300065308A0123206E308A01232075308A01B2
:100F400023200D308A0123200730BA000130B80079
:100F50005430AA004030AB008A010120E800680844
:100F6000A0006E308A013521B2006808A0006C3004
:100F70008A013021B4003208840034088A014A21F1
:100F80008A110A12031D5B2A8A01292F0730BA0031
:100F90000230B8005430AA004030AB00AE01AF01BF
:100FA0004E308A01232069308A01232076308A015D
:100FB000232065308A0123206C308A0123202030D1
:100FC0008A01232056308A0123206F308A01232092
:100FD0006C308A01232075308A0123206D308A010C
:100FE000232065308A0123206E308A01232020309F
:100FF0008A0123200230A9006A08A000A1010A305A
:10100000A200A3018A015121B2002108B3003208D5
:10101000A4003308A5002230B000B1018A01662087
:1010200020308A01232020308A0123202B308A019E
:1010300023202F308A0123202D308A0123202030C5
:101040008A01232056308A0123206F308A01232011
:101050006C308A01232075308A0123206D308A018B
:10106000232065308A0123206E308A01232020301E
:101070008A01232020308A0123206D308A01232019
:101080003D308A0123204D308A01232065308A01BA
:1010900023206E308A01232075308A0123200D30F1
:1010A0008A0123200730BA000130B8005430AA006A
:1010B0004030AB008A010120E800FA308A01EB20C1
:1010C0006808A0002C308A013521B2006808A00011
:1010D0002A308A013021B4003208840034088A01A1
:1010E0004A218A150A12031DA1286808A0002E3083
:1010F0008A013521B2006808A0002C308A01302115
:10110000B4003208840034088A014A218A150A1280
:10111000031DA8286808A0006E308A013521B2009E
:101120006808A0006C308A013021B40032088400C5
:1011300034088A014A218A110A12031D5B2A8A0196
:10114000C62F0A30EA078A150A1272268A01C62FAC
:101150000A30EA028A150A1272268A01C62F07305F
:10116000BA000230B8005430AA004030AB00AE01E3
:10117000AF014E308A01232069308A012320763066
:101180008A01232065308A0123206C308A012320C4
:1011900020308A01232053308A01232071308A01B4
:1011A000232075308A01232065308A0123206C308A
:1011B0008A01232063308A01232068308A0123209A
:1011C00020308A0123200230A9006908A000A10173
:1011D0000A30A200A3018A015121B2002108B30004
:1011E0003208A4003308A5002230B000B1018A0102
:1011F000662020308A01232020308A0123202B30D2
:101200008A0123202F308A0123202D308A012320B8
:1012100020308A01232053308A01232071308A0133
:10122000232075308A01232065308A0123206C3009
:101230008A01232063308A01232068308A01232019
:1012400020308A01232020308A0123206D308A013A
:1012500023203D308A0123204D308A012320653030
:101260008A0123206E308A01232075308A012320D1
:101270000D308A0123200730BA000130B800543005
:10128000AA004030AB008A010120E800FA308A0150
:10129000EB206808A0002C308A013521B2006808D4
:1012A000A0002A308A013021B400320884003408BA
:1012B0008A014A218A150A12031D8B296808A00099
:1012C0002E308A013521B2006808A0002C308A0136
:1012D0003021B4003208840034088A014A218A157A
:1012E0000A12031D93296808A0006E308A01352177
:1012F000B2006808A0006C308A013021B4003208C6
:10130000840034088A014A218A110A12031D5B2ACB
:101310008A150A12AF280A30E9078A150A127226BE
:101320008A150A12AF280A30E9028A150A127226B3
:101330008A150A12AF288711831687118312861720
:1013400083168613643083128A01EB205830C60757
:1013500003300318013EC7078A150A129C25071699
:101360008316071283128A150A12C0260730BA00A4
:101370000230B8005430AA004030AB00AE01AF01DB
:101380002A308A01232054308A01232058308A01D0
:1013900023202A308A01232020308A01232046304E
:1013A0008A01232072308A01232065308A0123209C
:1013B00063308A01232075308A01232065308A0139
:1013C00023206E308A01232063308A012320693074
:1013D0008A01232061308A01232020308A012320C2
:1013E0002D308A01232020308A0123200230A900D9
:1013F0006308A400A5012230B000B1018A01662073
:101400000430A9003E08A4003F08A5002230B00027
:10141000B1018A0166202E308A0123200130A90003
:101420004008A4004108A5002230B000B1018A01A3
:1014300066204D308A01232048308A0123207A30EB
:101440008A01232020308A01232020308A01232092
:1014500064308A0123203D308A01232064308A01D0
:10146000232065308A01232073308A0123207630BF
:101470008A01232069308A01232061308A012320D8
:1014800063308A01232069308A0123206F308A016A
:1014900023206E308A01232020308A0123207230DD
:1014A0008A0123203D308A01232052308A012320E3
:1014B00058308A01232020308A01232070308A018D
:1014C00023203D308A01232070308A0123206F3091
:1014D0008A01232074308A01232065308A01232069
:1014E0006E308A01232063308A01232069308A010B
:1014F000232061308A0123200A308A0123200D3005
:101500008A0123200730BA000130B8005430AA0005
:101510004030AB008A010120E8006808A000653077
:101520008A013521B2006808A00063308A013021A9
:10153000B4003208840034088A014A218A150A124C
:10154000031DEC2A6808A00073308A013521B2001F
:101550006808A00071308A013021B400320884008C
:1015600034088A014A218A150A12031DCF2A680805
:10157000A00071308A013521B2006808A0006F30E8
:101580008A013021B4003208840034088A014A21DB
:101590008A150A12031DF62B8A150A12B62907129C
:1015A000831607120A3083128A01EB2086138316F2
:1015B000861358308312C6020330031C013EC70253
:1015C0008A150A12952587158316871183128A15A5
:1015D0000A1272268A015B2A0730BA000230B8006C
:1015E0005430AA004030AB00AE01AF014E308A014A
:1015F000232069308A01232076308A012320653038
:101600008A0123206C308A01232020308A01232084
:1016100044308A01232065308A01232073308A01F7
:10162000232076308A01232069308A01232061300B
:101630008A01232063308A01232069308A01232014
:101640006F308A0123206E308A01232020308A01E6
:1016500023200230A9006208A000A1010A30A200E4
:10166000A3018A015121B2002108B3003208A4006D
:101670003308A5002230B000B1018A016620203075
:101680008A01232020308A0123202B308A01232045
:101690002F308A0123202D308A01232020308A0117
:1016A000232044308A01232065308A0123207330AF
:1016B0008A01232076308A01232069308A01232081
:1016C00061308A01232063308A01232069308A0136
:1016D00023206F308A0123206E308A01232020309E
:1016E0008A01232020308A01232078308A01232098
:1016F0003D308A0123204D308A01232065308A0144
:1017000023206E308A01232075308A012320203067
:101710008A01232054308A01232058308A01232053
:101720000A308A0123200D308A0123200730BA00B5
:101730000130B8005430AA004030AB008A010120CB
:10174000E800FA308A01EB206808A0002C308A01FA
:101750003521B2006808A0002A308A013021B40087
:101760003208840034088A014A218A150A12031DAE
:10177000E62B6808A0002E308A013521B2006808E7
:10178000A0002C308A013021B400320884003408D3
:101790008A014A218A150A12031DEE2B6808A0004F
:1017A00079308A013521B2006808A00077308A01BB
:1017B0003021B4003208840034088A014A218A1595
:1017C0000A12031DB6298A150A12EC2A0A30E2070A
:1017D0008A150A12C0268A150A12EC2A0A30E20279
:1017E0008A150A12C0268A150A12EC2A0730BA0096
:1017F0000230B8005430AA004030AB00AE01AF0157
:101800004E308A01232069308A01232076308A01F4
:10181000232065308A0123206C308A012320203068
:101820008A01232050308A0123206F308A0123202F
:1018300074308A01232065308A0123206E308A01AA
:10184000232063308A01232069308A0123206130FC
:101850008A01232020308A0123200230A900670852
:10186000A000A1010A30A200A3018A015121B20007
:101870002108B3003208A4003308A5002230B000CC
:10188000B1018A01662020308A01232020308A019C
:1018900023202B308A0123202F308A0123202D3052
:1018A0008A01232020308A01232050308A012320FE
:1018B0006F308A01232074308A01232065308A0129
:1018C00023206E308A01232063308A01232069306F
:1018D0008A01232061308A01232020308A012320BD
:1018E00020308A01232078308A0123203D308A016C
:1018F00023204D308A01232065308A0123206E3059
:101900008A01232075308A01232020308A01232078
:1019100054308A01232058308A0123200A308A015A
:1019200023200D308A0123200730BA000130B8008F
:101930005430AA004030AB008A010120E800FA30A0
:101940008A01EB206808A0002C308A013521B20002
:101950006808A0002A308A013021B40032088400CF
:1019600034088A014A218A150A12031DE42C6808EA
:10197000A0002E308A013521B2006808A0002C306A
:101980008A013021B4003208840034088A014A21D7
:101990008A150A12031DEC2C6808A00079308A0110
:1019A0003521B2006808A00077308A013021B400E8
:1019B0003208840034088A014A218A150A12031D5C
:1019C000B6298A150A12EC2A0A30E7078A150A1284
:1019D000C0268A150A12F62B0A30E7028A150A1267
:1019E000C0268A150A12F62B4608A0004708A10057
:1019F0002930A300D8308A0137218A110A12031D29
:101A00005B2A871183168711831286178316861324
:101A100028308312C60703300318013EC7078A1512
:101A20000A129C2507168316071283120730BA0084
:101A30000230B8005430AA004030AB00AE01AF0114
:101A40002A308A01232054308A01232058308A0109
:101A5000232020308A0123202D308A012320363094
:101A60008A01232030308A01232030308A0123204C
:101A70004B308A01232048308A0123207A308A01A2
:101A800023202A308A01232020308A01232020307D
:101A90008A01232072308A0123203D308A012320CD
:101AA00052308A01232058308A0123200A308A01CB
:101AB00023200D308A0123200730BA000130B800FE
:101AC0005430AA004030AB008A010120E8006808C9
:101AD000A00073308A013521B2006808A00071307F
:101AE0008A013021B4003208840034088A014A2176
:101AF0008A150A12031D7F2D8A150A12162D071248
:101B0000831607120A3083128A01EB20861383168C
:101B1000861328308312C6020330031C013EC7021D
:101B20008A150A1295258A015B2A8A150A12A025B0
:101B30008A150A121D2608008A150A12A025080017
:101B400086128316861206308312BA004030B8001F
:101B50000630BB001030B9000130B7006608A000A5
:101B6000A1018A0194208616831686120A308312F8
:101B70008A01EB2086128316861206308312BA0081
:101B80004030B8000630BB001030B9000130B7005B
:101B90004408A0004508A1000F308A019520861650
:101BA000831686120A3083128A01EB20861283166E
:101BB00086128312061683160612831206128316E5
:101BC000061206308312BA004030B8000630BB005F
:101BD0001030B9000130B7004608A0004708A10046
:101BE0000F308A01952086168316861283124608C6
:101BF000A0004708A1006430A200A3018A0151217E
:101C0000E4004608A0004708A1006430A200A30138
:101C10008A0151212408E50003178D01031364088C
:101C20008A01DD20031701308D00031365088A0146
:101C3000DD2032308A01EB2008000E30E3005830FE
:101C40004607B20003300318013E4707B300A03037
:101C5000B2022830031C013EB3023208A60033084A
:101C6000A7001930A200A3018A016D21B200250846
:101C7000B3000310330CBF00320CBE0058304607CF
:101C8000B20003300318013E4707B300A030B20290
:101C90002830031C013EB3023208A6003308A70017
:101CA0001930A200A3018A016D21B2002508B300FA
:101CB0003208A0003308A1000230A200A3018A016B
:101CC00051212408B2002508B3003208A6003308C9
:101CD000A7000530A200A3018A016D21C0002508DC
:101CE000C1000800871783168713013083128A0109
:101CF000EB200717831607138312871683168712A4
:101D00008312871283168712831207138316071311
:101D100007308312BA002030B8000730BB004030D3
:101D2000B9000130B7006A08A000A1018A0194201F
:101D30000730BA002030B8000730BB004030B9008F
:101D40000130B7006908A000A1018A019420013088
:101D50008A01EB208713831687138312031702303F
:101D60008D0003136A088A01DD20031703308D00FC
:101D7000031369088A01DD2005308A01EB20080081
:101D8000061583160611013083128A01EB20861591
:101D9000831686118312861483168610831286108A
:101DA00083168610831286118316861106308312DD
:101DB000BA000230B8000630BB000830B90001306C
:101DC000B7006208A000A1018A0194200630BA0081
:101DD0000230B8000630BB000830B9000130B7004F
:101DE0006708A000A1018A01942001308A01EB203C
:101DF0000611831606118312031704308D00031396
:101E000062088A01DD20031705308D00031367087F
:101E10008A01DD2005308A01EB20080063008A1565
:041E20000A120E2F65
:02400E00753DFE
:00000001FF
